:020000040000FA
:040000008EEF1AF075
:08000800056ED8CF06F0E0CF31
:1000100007F00001E9CF0DF0EACF08F0E1CF09F0D9
:10002000E2CF0AF0D9CF0BF0DACF0CF0F3CF14F017
:10003000F4CF15F0FACF16F000C00FF001C010F0A9
:1000400002C011F003C012F004C013F0F2AA2CEFAA
:1000500000F0F2B47FEF01F00FC000F010C001F02B
:1000600011C002F012C003F013C004F00E8E0DC0D8
:10007000E9FF08C0EAFF09C0E1FF0AC0E2FF0BC0C8
:10008000D9FF0CC0DAFF14C0F3FF15C0F4FF16C08F
:10009000FAFF055007C0E0FF06C0D8FF1000F2CFFE
:1000A0000EF0F29EF76AB80FF66E000EF722090006
:1000B000F5500EBEF28E1200008040C020A060E01D
:1000C000109050D030B070F0088848C828A868E870
:1000D000189858D838B878F8048444C424A464E440
:1000E000149454D434B474F40C8C4CCC2CAC6CEC10
:1000F0001C9C5CDC3CBC7CFC028242C222A262E210
:10010000129252D232B272F20A8A4ACA2AAA6AEA0F
:100110001A9A5ADA3ABA7AFA068646C626A666E6DF
:10012000169656D636B676F60E8E4ECE2EAE6EEEAF
:100130001E9E5EDE3EBE7EFE018141C121A161E1C7
:10014000119151D131B171F1098949C929A969E9DF
:10015000199959D939B979F9058545C525A565E5AF
:10016000159555D535B575F50D8D4DCD2DAD6DED7F
:100170001D9D5DDD3DBD7DFD038343C323A363E37F
:10018000139353D333B373F30B8B4BCB2BAB6BEB7F
:100190001B9B5BDB3BBB7BFB078747C727A767E74F
:1001A000179757D737B777F70F8F4FCF2FAF6FEF1F
:1001B0001F9F5FDF3FBF7FFF0DAE03D0F2CF0EF07A
:1001C000F29EF76ADA0FF66E010EF7220900F5507B
:1001D0000DAE02D00EBEF28E120000102030405044
:1001E00060700000000000000000F2CF0EF0F29EF0
:1001F000F76A040FF66E020EF7220900F5500EBEE4
:10020000F28E12002530344C58303030310002016B
:10021000556B566B92948994C950610EC96EC73064
:10022000FEE3C950C96AC730FEE3C950036A556F7F
:1002300003C056F255C203F0000E556F03C056F2CC
:10024000C950C96AC730FEE3C95055135631036E11
:100250005531026E033202323F0E031602C055F2D0
:1002600003C056F2000B006E5651200B036E005077
:10027000031002E0C00E561355C201F056C202F040
:10028000000144EF01F0C3D702C054F201C053F2A1
:10029000020153C201F054C202F00001000C92941A
:1002A00089940201555180095611586FC95058C29E
:1002B000C9FFC730FEE3929489840001000C02015B
:1002C0005151020802E1516B09D0515303E1010E73
:1002D000516F04D0512D02D0020E516F036A52515A
:1002E000F2CF53F2F29E000167DF020153BFF28E9C
:1002F000546F51C255F2566F0001D1DF000CEC5122
:10030000EA250201516F0001ED51EB210201D76E88
:1003100051C2D6FF0001EE2BD8B4EF2BED6BEC6B86
:10032000EF5303E1EE51020805E2EF6BEE6BED6B6C
:10033000140EEC6FDF2BE851DF5D15E1E95313E19B
:10034000DF6BDE2BDE510A080EE1DE6BDD2BDD51AB
:100350003C0809E1DD6BDC2BDC513C0804E1DC6B83
:10036000DA2BD8B4DB2B0101E62D91D0E75327E13E
:10037000D890E035026EE135036E0250F00F016E49
:10038000000E032201C051F203C052F200017BDFD4
:1003900052C2EAFF51C2E9FF02C0ECFFED5201C0B8
:1003A000EFFF010E0101E76F0201516FE8C152F248
:1003B000000185DF0101E02BD8B4E12B51D0E72DFE
:1003C00027D0D890E035026EE135036E0250F00F71
:1003D000016E000E032201C051F203C052F200016F
:1003E00052DF52C2EAFF51C2E9FF02C0ECFFED52F8
:1003F00001C0EFFF020E0101E76F0201516FE9C179
:1004000052F200015CDF0101E02BD8B4E12B28D0CF
:10041000E751020825E1D890E035026EE135036E20
:100420000250F00F016E000E032201C051F203C012
:1004300052F2000128DF52C2EAFF51C2E9FF02C0B6
:10044000ECFFED5201C0EFFF0101E76B0201516BC0
:10045000E8C152F2000133DF0101E02BD8B4E12BF7
:10046000E0513C0808E1E15306E1E56BE46BE36B26
:10047000010EE26F0CD0E051780809E1E15307E189
:10048000E56BE46BE36B020EE26FE16BE06BF29401
:1004900000012CEF00F0020EEA6EE96AEF500EE068
:1004A0000C0E016E006A002EFED7012EFBD7F70E50
:1004B000006E002EFED700D0EF2EF2D7000CEBC05E
:1004C000D7FFEAC0D6FF020100C2E9FF01C2EAFF7E
:1004D000EC6AED52EF6A020E0025E96E000E012172
:1004E000EA6EEF6A030E0025E96E000E0121EA6E46
:1004F000EF6A040E0025E96E000E0121EA6EEF6A34
:10050000050E0025E96E000E0121EA6EEF6A00017A
:10051000000C92948994C950180EC96EC730FEE33E
:10052000C950C96AC730FEE392948984ADEF02F0E6
:1005300092948994FEC100F20201C950FEC1C9FF24
:10054000C730FEE3C950FFC1C9FFC730FEE3929434
:1005500089840001B4EF02F0DCD7070E0101FE6FC1
:100560003E0EFF6F0001E4D792908990EDEF0EF000
:10057000016A026A006A036A02010D5102E10C512C
:1005800018E0100E0E6FD8900A370B37003603367E
:100590000D51035C02E10C51005C07E30C51005E5D
:1005A000D8A003060D51035ED880013602360E2F07
:1005B000EAD700014EEF0DF08E0E006E2EC201F054
:1005C0002DC202F0036A015209E102C001F0026A81
:1005D000080E005E015202E1006A08D0D89001BE08
:1005E00004D0023601360006F9D7019E000C3EC247
:1005F00045F202014251451B45AF05D0D894D89031
:100600003EBFD8802FD03EC245F241C246F23D5196
:10061000465F06E045AF26D0D850010AD86E22D0FA
:1006200042C246F23E51465F06E045AF1BD0D8506D
:10063000010AD86E17D043C246F23F51465F06E02A
:1006400045AF10D0D850010AD86E0CD044C246F243
:100650004051465F06E045AF05D0D850010AD86E3C
:1006600001D0D8900001000C800ED8A202D0020167
:10067000461B02014B6B4C6B42C24AF246514A1B6D
:100680004151D8B4DFD0496F006E4551D8B4E3D0A2
:10069000495FD8B483D03EE346C24FF24F8F47C282
:1006A0004EF248C24DF24C6BD8904F334E334D331F
:1006B0004C33492FF8D74AAF03D04B81E0D04B9150
:1006C00049914B89020EEA6E440EE96EEBD04B99CC
:1006D0004ABF0AD049A113D04F334E334D334C3368
:1006E000002AD8B4C7D00BD04FBF0CD0D8904C370D
:1006F0004D374E374F370006D8B4BCD0F5D74B8DA9
:100700006DD04B9D42C24AF242AF02D04F8FABD068
:100710004F9FA9D045C249F245C200F04151495FFF
:1007200042C24FF24F8F43C24EF244C24DF24C6B65
:10073000D8904F334E334D334C33492FF8D74AAF0F
:1007400003D04B839CD04B9349914B8B020EEA6EA6
:10075000480EE96EA7D04B9B4ABF0AD049A113D0DF
:100760004F334E334D334C33002AD8B483D00BD0A3
:100770004FBF0CD0D8904C374D374E374F3700060F
:10078000D8B478D0F5D74B8F29D04B9F46C24AF2C8
:1007900046AF02D04F8F67D04F9F65D046C24FF211
:1007A0004F8F47C24EF248C24DF24AAF04D04F9F1E
:1007B0004B8565D04B954C6B4991020EEA6E440E09
:1007C000E96E70D04ABF1CD042C24AF249A106D09D
:1007D0004F334E334D334C33002A4CE04CAF0BD0EB
:1007E0004D2B09E14E2B07E14F2B05E14F334E33E3
:1007F0004D33002A3FE04BBD84D74BBFC6D71CD03A
:10080000800E4F1B4FAF04D03AD046C24AF20AD0F6
:1008100042C24AF24F5306E14E5304E14D5302E106
:10082000006A21D04FBF08D0D8904C374D374E3793
:100830004F37002EF7D71ED04AAF02D04F8F13D0BC
:100840004F9F11D045C200F046C24FF247C24EF250
:1008500048C24DF208D041C200F042C24FF243C23A
:100860004EF244C24DF24FC201F04EC202F04DC2F0
:1008700003F034D0006A016A026A036A2FD04C6B1D
:100880004D1F4E1F4F1F4C1F4C2B05E14D2B03E1FD
:100890004E2B01E14F2B4BB112D74BB354D74BB575
:1008A00089D7B3D7EF504D2705E34E2B03E14F2BEC
:1008B000D8B44981ED52EF504E2703E34F2BD8B403
:1008C0004981ED52EF50EFBE01D0800A4F27D8B0DA
:1008D00049814BB9FCD64BBB3ED774D70001000C05
:1008E00002014151D8B4A5D04D6F4551D8B4A1D023
:1008F0004D5F05E37F0E4D27D8B09BD006D0810E0B
:100900004D5FD8A096D0D8B494D04DC200F0016A03
:10091000026A036A4C6B42C24BF24B8F43C24AF2EB
:1009200044C249F2190E4D6F4851495F0DE2010E64
:100930004A5F0AE24B5F08E24C5F06E24C2B4B2B0E
:100940004A2B4851492728D047514A5F12E2010EED
:100950004B5F0FE24C5F0DE24C2B4B2B47514A276C
:100960004851492719E34A2B17E14B2B15E14C2B32
:1009700013D0465180094B5F0EE2010E4C5F0BE233
:100980004C2B465180094B2747514A27E9E34B2B13
:10099000E7E14C2BE5D703804D2F01D00BD0D89049
:1009A00049374A374B374C37D89003360236013631
:1009B0004E37BAD74EA106D0D89001320232033258
:1009C0004E3302D0000635E04EBF1ED0D8904937D6
:1009D0004A374B374C374851495F07E2010E4A5FAF
:1009E00004E24B5F02E24C5F1AE347514A5F05E2C3
:1009F000010E4B5F02E24C5F12E3465180094B5FF0
:100A000003E2010E4C5F0BE3032A09E1022A07E12E
:100A1000012A05E1002A0DE001320232033242C20E
:100A20004DF246514D1B4DAF02D0018E06D0019EB6
:100A300004D0006A016A026A036A0001000C020124
:100A40003D51D8B471D0006E4151D8B46DD000265C
:100A500004E3810E002668E204D07F0E005E64E3AA
:100A600063E03EC245F24251451B3E8F428F4051EA
:100A70004403F4CF47F23F514303F4CF03F0F3CFE5
:100A800046F24403F3504727F4504623000E032256
:100A900040514303F3504727F4504623000E026AA7
:100AA000032202223E514403F3504627F45003220E
:100AB000000E02223E514303F3500326F45002225B
:100AC000000E016A012240514203F3504627F450C0
:100AD0000322000E022201223F514203F35003265B
:100AE000F4500222000E01223E514203F35002262E
:100AF000F4500122002A01BE05D0463703360236E3
:100B000001360006000E46AF0AD0032A0222012257
:100B1000015005E1025003E1035001E1002A45BF05
:100B2000018E45AF019E04D0006A016A026A036A21
:100B30000001000C8E0E006E40C201F03FC202F0B8
:100B4000036A01AE05D0011E021E022A01E1012A3C
:100B5000015209E102C001F0026A080E005E015272
:100B600002E1006A0DD0D89001BE04D002360136F1
:100B70000006F9D7020140AF02D0000101D0019E6A
:100B80000001000C2BC22FF22AC22EF229C22DF234
:100B900028C22CF22FC240F22EC23FF22DC23EF2EA
:100BA0002CC23DF20201446B436B426B7F0E416FDE
:100BB00000011DDDD8B435D2020E02013E6F2C0EAD
:100BC000E96E3EC2EAFF7E0EEF6ED8822FC244F27B
:100BD0002EC243F22DC242F22CC241F2486B476B47
:100BE000466B7F0E456F00013FDD00C03DF201C046
:100BF0003EF202C03FF203C040F2D8922FC244F24C
:100C00002EC243F22DC242F22CC241F20201486BC5
:100C1000476B466B7F0E456F000126DD40C244F2F4
:100C20003FC243F23EC242F23DC241F203C048F22B
:100C300002C047F201C046F200C045F251DE03C0D7
:100C40002FF202C02EF201C02DF200C02CF22FC2F2
:100C500040F22EC23FF22DC23EF22CC23DF22FC214
:100C600044F22EC243F22DC242F22CC241F2E7DE20
:100C700003C03BF202C03AF201C039F200C038F2C0
:100C8000BC0E0201406F240E3F6F670E3E6F7D0E5B
:100C90003D6F3BC244F23AC243F239C242F238C21B
:100CA00041F20001CCDE00C03DF201C03EF202C0C4
:100CB0003FF203C040F2D89203C044F202C043F2B4
:100CC00001C042F200C041F2E30E0201486FE40E9F
:100CD000476F900E466F820E456F0001C5DC03C062
:100CE00033F202C032F201C031F200C030F233C23E
:100CF00040F232C23FF231C23EF230C23DF23BC25C
:100D000044F23AC243F239C242F238C241F297DEAB
:100D100000C03DF201C03EF202C03FF203C040F20B
:100D2000D89203C044F202C043F201C042F200C0B4
:100D300041F21C0E0201486F870E476F570E466F37
:100D4000830E456F000190DC03C033F202C032F223
:100D500001C031F200C030F233C240F232C23FF281
:100D600031C23EF230C23DF23BC244F23AC243F2DB
:100D700039C242F238C241F262DE00C03DF201C027
:100D80003EF202C03FF203C040F2D89203C044F2E8
:100D900002C043F201C042F200C041F2AB0E0201B8
:100DA000486FE10E476F9E0E466F830E456F000140
:100DB0005BDC03C033F202C032F201C031F200C08A
:100DC00030F20201406B3F6B3E6B7F0E3D6F3BC2CA
:100DD00044F23AC243F239C242F238C241F200014F
:100DE0002EDE00C03DF201C03EF202C03FF203C061
:100DF00040F2D89203C044F202C043F201C042F272
:100E000000C041F2B40E0201486F2A0E476F820EF5
:100E1000466F456F000128DC03C037F202C036F28E
:100E200001C035F200C034F237C240F236C23FF2A0
:100E300035C23EF234C23DF23BC244F23AC243F202
:100E400039C242F238C241F2FADD00C03DF201C0BF
:100E50003EF202C03FF203C040F2D89203C044F217
:100E600002C043F201C042F200C041F2800E020112
:100E7000486F3E0E476F060E466F830E456F0001AA
:100E800034EC03F003C037F202C036F201C035F291
:100E900000C034F237C240F236C23FF235C23EF2F1
:100EA00034C23DF23BC244F23AC243F239C242F28A
:100EB00038C241F2C4DD00C03DF201C03EF202C0C2
:100EC0003FF203C040F2D89203C044F202C043F2A2
:100ED00001C042F200C041F2AB0E0201486FE10EC8
:100EE000476F9E0E466F820E456F000134EC03F093
:100EF00003C037F202C036F201C035F200C034F24E
:100F00002FC240F22EC23FF22DC23EF22CC23DF261
:100F100033C244F232C243F231C242F230C241F231
:100F20008EDD00C03DF201C03EF202C03FF203C0C0
:100F300040F203C044F202C043F201C042F200C0DA
:100F400041F237C248F236C247F235C246F234C2E5
:100F500045F2C6DC03C033F202C032F201C031F206
:100F600000C030F2020E02013E6F280EE96E3EC252
:100F7000EAFF7E0EEF5C3C6F3CBF01D014D0000E48
:100F8000D8803C55406B3F6F3FBF40070001D2DD2A
:100F900000C034F20150800A0201356F02C036F2FF
:100FA00003C037F210D0406B3CC23FF23FBF400756
:100FB0000001C0DD03C037F202C036F201C035F2D5
:100FC00000C034F2020137C240F236C23FF235C2ED
:100FD0003EF234C23DF2180E446F720E436F310E72
:100FE000426F7E0E416F00012ADDD89233C244F277
:100FF00032C243F231C242F230C241F203C048F27F
:1010000002C047F201C046F200C045F234EC03F0E2
:1010100003C033F202C032F201C031F200C030F23C
:1010200006D00201336B326B316B306B000130C282
:1010300000F031C201F032C202F033C203F0000C02
:1010400011C22BF210C22AF20FC229F20EC228F2EC
:1010500099DD03C015F202C014F201C013F200C002
:1010600012F215C244F214C243F213C242F212C287
:1010700041F28E0E0201486F5D0E476F130E466FF0
:10108000800E456F00012CDC03C015F202C014F283
:1010900001C013F200C012F212C200F013C201F03C
:1010A00014C202F015C203F067EF0DF08E0E006E51
:1010B00002013B51005E3CC202F03DC201F0028ED3
:1010C000005209E0D890025202E1015204E00232DB
:1010D0000132002EF7D73CAF05D0011E021E012AB7
:1010E000D8B4022A0001000C020128911CC221F28E
:1010F0001BC220F21AC21FF219C21EF21CC240F219
:101100001BC23FF21AC23EF219C23DF2446B436B5E
:10111000426B416B0001F7EC02F005E3020128810C
:101120001F51800A1F6F21C240F220C23FF21FC22E
:101130003EF21EC23DF20201446B436B426B8E0EC7
:10114000416F0001F7EC02F001E218E121C23EF22A
:1011500020C23DF21FC23CF21EC23BF2A7DF02C01A
:101160002EF201C02DF2DCEC02F003C025F202C029
:1011700024F201C023F200C022F2D1D021C240F2F9
:1011800020C23FF21FC23EF21EC23DF2800E02019B
:10119000446F960E436F180E426F960E416F00011A
:1011A000F7EC02F0D8A0B3D021C244F220C243F23F
:1011B0001FC242F21EC241F20201486B476B466BEE
:1011C0008E0E456F000170EC04F003C03EF202C0C9
:1011D0003DF201C03CF200C03BF268DF02C027F2E2
:1011E00001C026F221C244F220C243F21FC242F2E1
:1011F0001EC241F20201486B476B466B8E0E456F73
:10120000000170EC04F000C029F201C02AF202C013
:101210002BF203C02CF227C22EF226C22DF2DCECF8
:1012200002F0D8822CC244F22BC243F22AC242F20C
:1012300029C241F203C048F202C047F201C046F29F
:1012400000C045F234EC03F00201406B3F6B3E6B93
:101250008E0E3D6F03C044F202C043F201C042F261
:1012600000C041F200011FEC05F003C021F202C0F2
:1012700020F201C01FF200C01EF227C22EF226C2C9
:101280002DF2DCEC02F00201406B3F6B3E6B8E0EE8
:101290003D6F03C044F202C043F201C042F200C0FD
:1012A00041F200011FEC05F003C025F202C024F258
:1012B00001C023F200C022F221C23EF220C23DF260
:1012C0001FC23CF21EC23BF2F1DE02C02EF201C090
:1012D0002DF2DCEC02F0D89225C244F224C243F293
:1012E00023C242F222C241F203C048F202C047F2D6
:1012F00001C046F200C045F234EC03F003C025F211
:1013000002C024F201C023F200C022F208D021C2A0
:1013100025F220C224F21FC223F21EC222F221C2F1
:101320003EF220C23DF21FC23CF21EC23BF2BEDEC4
:1013300002C02EF201C02DF2DCEC02F0D88221C2F4
:1013400044F220C243F21FC242F21EC241F203C065
:1013500048F202C047F201C046F200C045F234EC48
:1013600003F003C021F202C020F201C01FF200C04E
:101370001EF2020128A103D02351800A236F21C24B
:1013800040F220C23FF21FC23EF21EC23DF2446B49
:10139000436B426B416B0001F7EC02F03CE0020151
:1013A00028A11CD01D531AE1D88225C244F224C2C0
:1013B00043F223C242F222C241F2486B476B466BB2
:1013C0007F0E456F000134EC03F003C025F202C02C
:1013D00024F201C023F200C022F2020128B11CD085
:1013E0001D2D1AD0D89225C244F224C243F223C242
:1013F00042F222C241F2486B476B466B7F0E456F4B
:10140000000134EC03F003C025F202C024F201C055
:1014100023F200C022F202011CC240F21BC23FF2C2
:101420001AC23EF219C23DF2446B436B426B416BF0
:101430000001F7EC02F006E10201256B246B236B3F
:10144000226B000122C200F023C201F024C202F08C
:1014500025C203F038EF0AF018C21CF217C21BF2C3
:1014600016C21AF215C219F202011D6B00013CD618
:10147000000C2CC244F22BC243F22AC242F229C20F
:1014800041F2180E0201486F720E476F310E466F1F
:101490007E0E456F000170EC04F003C03EF202C006
:1014A0003DF201C03CF200C03BF200DE01C039F267
:1014B00002013A912CC230F22BC22FF22AC22EF234
:1014C00029C22DF22CC240F22BC23FF22AC23EF2B8
:1014D00029C23DF2446B436B426B416B0001F7EC58
:1014E00002F006E302013A81396D2E51800A2E6F17
:1014F0000201346B336B326B316B020E3C6F310E79
:10150000E96E3CC2EAFF7F0E3925EF6E30C244F22D
:101510002FC243F22EC242F22DC241F2180E486F82
:10152000720E476F310E466F7E0E456F000170ECF4
:1015300004F000C03BF201C03CF202C03DF203C027
:101540003EF20201406B39C23FF23FBF400700014B
:101550009AEC05F0D8823EC244F23DC243F23CC24E
:1015600042F23BC241F203C048F202C047F201C05E
:1015700046F200C045F234EC03F003C030F202C082
:101580002FF201C02EF200C02DF27C0E0201406F3E
:10159000880E3F6F590E3E6F720E3D6F30C244F29F
:1015A0002FC243F22EC242F22DC241F200011FECC3
:1015B00005F000C03BF201C03CF202C03DF203C0A6
:1015C0003EF2D89203C044F202C043F201C042F29C
:1015D00000C041F2E00E0201486F970E476F260EE1
:1015E000466F750E456F000134EC03F003C038F20E
:1015F00002C037F201C036F200C035F238C240F204
:1016000037C23FF236C23EF235C23DF230C244F23A
:101610002FC243F22EC242F22DC241F21FEC05F05E
:1016200000C03BF201C03CF202C03DF203C03EF2FA
:10163000D89203C044F202C043F201C042F200C09B
:1016400041F2C40E0201486F1D0E476F1E0E466F19
:10165000780E456F000134EC03F003C038F202C08D
:1016600037F201C036F200C035F238C240F237C25C
:101670003FF236C23EF235C23DF230C244F22FC2D2
:1016800043F22EC242F22DC241F21FEC05F000C01F
:101690003BF201C03CF202C03DF203C03EF2D892E0
:1016A00003C044F202C043F201C042F200C041F262
:1016B0005E0E0201486F500E476F630E466F7A0E42
:1016C000456F000134EC03F003C038F202C037F27A
:1016D00001C036F200C035F238C240F237C23FF2E4
:1016E00036C23EF235C23DF230C244F22FC243F25E
:1016F0002EC242F22DC241F21FEC05F000C03BF2B7
:1017000001C03CF202C03DF203C03EF2D89203C0D9
:1017100044F202C043F201C042F200C041F21A0E8C
:101720000201486FFE0E476F750E466F7C0E456FC7
:10173000000134EC03F003C038F202C037F201C0FC
:1017400036F200C035F238C240F237C23FF236C23C
:101750003EF235C23DF230C244F22FC243F22EC2F5
:1017600042F22DC241F21FEC05F000C03BF201C075
:101770003CF202C03DF203C03EF2D89203C044F2F4
:1017800002C043F201C042F200C041F2180E020151
:10179000486F720E476F310E466F7E0E456F000127
:1017A00034EC03F003C038F202C037F201C036F265
:1017B00000C035F230C240F22FC23FF22EC23EF2DC
:1017C0002DC23DF238C244F237C243F236C242F271
:1017D00035C241F21FEC05F0D8920201446B436B15
:1017E000426B7F0E416F03C048F202C047F201C056
:1017F00046F200C045F2000134EC03F034C240F27E
:1018000033C23FF232C23EF231C23DF203C044F273
:1018100002C043F201C042F200C041F21FEC05F0E9
:1018200003C034F202C033F201C032F200C031F220
:1018300002013AA119D0446B436B426B7F0E416F9A
:1018400034C248F233C247F232C246F231C245F2E4
:10185000000170EC04F003C034F202C033F201C0A6
:1018600032F200C031F2020131C200F032C201F0A6
:1018700033C202F034C203F00001000C0201406BDD
:101880003F6B3E6B3D6B1FC244F21EC243F21DC252
:1018900042F21CC241F20001F7EC02F001E22FE13A
:1018A0001FC22BF21EC22AF21DC229F21CC228F24C
:1018B000C2EC05F023C240F222C23FF221C23EF246
:1018C00020C23DF203C044F202C043F201C042F222
:1018D00000C041F21FEC05F000C024F201C025F267
:1018E00002C026F203C027F203C02CF202C02BF282
:1018F00001C02AF200C029F2BCDD3BD03AD01CC2A4
:1019000024F202011D51800A256F1EC226F21FC259
:1019100027F21FC22BF21EC22AF2296F1CC228F224
:101920000001C2EC05F023C240F222C23FF221C204
:101930003EF220C23DF203C044F202C043F201C0B5
:1019400042F200C041F21FEC05F000C025F201C0D8
:1019500026F202C027F203C028F203C02CF202C014
:101960002BF201C02AF200C029F283DD800E011A99
:1019700000D0E2EF0CF0800E0201146F156B166BB5
:10198000176B406B13C23FF23FBF400700019AEC58
:1019900005F000C018F201C019F202C01AF203C02B
:1019A0001BF217C21FF216C21EF215C21DF214C29C
:1019B0001CF203C023F202C022F201C021F200C0D7
:1019C00020F25CD712C240F211C23FF210C23EF2C6
:1019D0000FC23DF203C044F202C043F201C042F222
:1019E00000C041F21FEC05F0B3EF0DF0080E016EE0
:1019F0000A0E006E0400002EFDD78B9094900A0E04
:101A0000006E0400002EFDD702010D378B92D8B076
:101A10009482D8A09492948082A0FED7012E01D007
:101A200002D00001E5D70A0E006E0400002EFDD79B
:101A30008B909490000094820A0E006E0400002E99
:101A4000FDD70A0E006E0400002EFDD7948082A000
:101A5000FED7016A0A0E006E0400002EFDD782B286
:101A600001808B9094908B9294920001000C020163
:101A70000551040808E303E104510E0804E3040ED1
:101A8000056F0F0E046F05C20BF204C20AF2040EBA
:101A90000D6F0F0E0C6F0001B8EF02F002C02EF2B6
:101AA00001C02DF20001DCEC02F000C00AF201C01E
:101AB0000BF202C00CF203C00DF203C011F202C01F
:101AC00010F201C00FF200C00EF220EF08F0A60ED7
:101AD0000201406F9B0E3F6F540E3E6F800E3D6FB4
:101AE00003C044F202C043F201C042F200C041F21E
:101AF00000011FEC05F000C00BF201C00CF202C0A7
:101B00000DF203C00EF203C018F202C017F201C0BA
:101B100016F200C015F2A0DC03C03EF202C03DF296
:101B200001C03CF200C03BF256EC08F001C007F2E5
:101B3000020107510F0802E20F0E076F8A0E0A6FAB
:101B4000010E0B6FE00E0C6F0D6B0A0E07250E6F6A
:101B50000DC212F20CC211F20BC210F20AC20FF245
:101B6000136F000108D700C00BF201C00CF202C0D5
:101B70000DF203C00EF205C22EF204C22DF2DCEC0F
:101B800002F00EC244F20DC243F20CC242F20BC28A
:101B900041F203C048F202C047F201C046F200C061
:101BA00045F270EC04F0EACF10F2E9CF0FF2D882E0
:101BB0000201446B436B426B8A0E416F03C048F2D3
:101BC00002C047F201C046F200C045F2000134EC09
:101BD00003F010C2EAFF0FC2E9FF00C011F201C01A
:101BE00012F202C013F203C014F203C018F202C0D2
:101BF00017F201C016F200C015F22EDC03C03EF24F
:101C000002C03DF201C03CF200C03BF256EC08F0CD
:101C100002C009F201C008F20201073BF00E0717EB
:101C20000837093708370937FC0E0817020E0B6F03
:101C3000080E0A6F010E0A25016E000E0B2101C06D
:101C4000E9FFEA6EEF500711EF6E020E036E080E09
:101C5000E96E03C0EAFFEF50FC0B006E036A005010
:101C6000ED52EF6E03C0ECFF020E036E080EE96E3C
:101C700003C0EAFFEF500611006EECCF03F00050F6
:101C8000ED52EF6E03C0ECFF94820A0E006E04006A
:101C9000002EFDD794800A0E006E0400002EFDD7A2
:101CA0008B9294920A0E006E0400002EFDD78B904A
:101CB00094900351FE0B0A6F0D6F000197DE020E28
:101CC00002010B6F080E0A6F010E0A25016E000E4D
:101CD0000B21036E01C0E9FFEA6EEFCF0CF20CC2DC
:101CE0000DF2000183DE020E036E080EE96E03C0E2
:101CF000EAFFECCF0BF2ED52EFCF0AF20AC20DF27F
:101D000075DE94920000948082A0FED70A0E006EC9
:101D10000400002EFDD700D0000094820A0E006E51
:101D20000400002EFDD7000C0201005102080BE157
:101D30002E0E036F02C205F201C204F2066B00010F
:101D400096DE0AD002012C0E036F02C205F201C218
:101D500004F2066B00018BDE000CD96BD791000CEE
:101D6000B0989484BD6A796A9482BA6A676AC150ED
:101D7000C00B0F09C16EC290929A899A020E01019E
:101D8000FE6FFA0E0201006F00014BEC02F0010140
:101D9000FE2FF7D7010EEF6F900EEE6F0001E96B8B
:101DA000780EE86FFB0EEB6FEE0EEA6FED6BEC6BEF
:101DB000EF6BEE6B820ED56E0201016BDA0E006FD7
:101DC00000015FEC02F0C69A949A94889496210ED2
:101DD000C66E000EC76EACEF02F00101E86BE96B56
:101DE000090EEB6FC40EEA6F270EED6F100EEC6F4D
:101DF000186AF2BE188EF29E0201516BE8C152F2CF
:101E000000015FEC01F018BEF28E0101E76B0201E8
:101E1000006BEBC102F2EAC101F2000185DF020EA4
:101E20000201006FEDC102F2ECC101F200017CDFA2
:101E300094DF96928D8296908D800101E66BE56B22
:101E4000E46BE36BE26BE16BE06BF36B010EF26F43
:101E5000F16BF06FC00EF2129298899898948F846B
:101E6000F46BF66BF56B9886F76B86B6F72B000173
:101E7000B1EF1AF00201036B988286B216D09692E7
:101E80008D92060E006E002EFED70000FF0E956E9E
:101E90008350F2CF05F2F29E00014FEC00F00201F8
:101EA00005BFF28E036F96928D8203C201F000018E
:101EB0002FEF10F002010C6B0D6B0E6B0F6B0B6BA9
:101EC0000A510B5D5EE20C370D370E370F370C37BA
:101ED0000D370E370F370C370D370E370F370C37DE
:101EE0000D370E370F37F00E0C17036A0B5108250C
:101EF000E96E09510320EA6EEF50390820E3036AC6
:101F00000B510825E96E09510320EA6EEF500C25AC
:101F1000106F000E0D21116F000E0E21126F000EBA
:101F20000F21136F300E105D0C6F000E11590D6FE5
:101F3000000E12590E6F000E13590F6F20D00A0EAB
:101F40000C25106F000E0D21116F000E0E21126F67
:101F5000000E0F21136F036A0B510825E96E09511A
:101F60000320EA6E410EEF5C10250C6F000E11216C
:101F70000D6F000E12210E6F000E13210F6F0B2B31
:101F80009FD70CC200F00DC201F00EC202F00FC2CA
:101F900003F00001000C0201016B026B1B500208F0
:101FA00003E0000E016E43D0010E0001D85D036A0C
:101FB0001B0FE96E000E0320EA6EEF50030804E0E9
:101FC000000E016E020133D0010E0201036F030EF9
:101FD0000001D85D0201035D0BE2036A03511B0F90
:101FE000E96E000E0320EA6EEF500127032BEFD7B6
:101FF000011F030E0001D85D036A1B0F0201066F6B
:10200000000E0320076F096F06C208F2020E0A6F66
:10201000000150DF00C002F202010151025D04E044
:10202000000E016E04D003D0010E016E00D000013D
:1020300051EF10F092DE0201006B00513F0827E3E0
:10204000988286B221D0036A00511B0F016E000EE8
:10205000032201C001F203C002F200010BD702C249
:10206000EAFF01C2E9FF01C0EFFF036A020100516C
:102070001B0FE96E000E0320EA6EEF50030803E128
:1020800000C2D9F004D001D002D0002BD6D7000175
:10209000D9513F080CE3D7B109D0010ED925D86F2B
:1020A0007AD7015202E0D78101D057DE01D055DE48
:1020B000BAEF1AF0FAC1EAFFF9C1E9FF020107C25B
:1020C000EFFFE92AD8B4EA2AEF6A0101F92BD8B464
:1020D000FA2B0001000C020106BF11D00F0E006E9A
:1020E000053900160A0E005C03E2300E002602D00D
:1020F0000651002600C007F20001DCDF02010F0ECE
:1021000005170A0E055D02E2300E02D0069F065149
:10211000052705C207F20001CDDF000C0201036BA9
:10212000035177080BE3036A03515B0FE96E000E5E
:102130000320EA6EFF0EEF6E032BF2D700C200F011
:102140000151036E05E100520001D8B4E3D0020151
:10215000035006E1010E005C0001D8B4ECD002018E
:10216000035006E1020E005C0001D8B4F6D0020173
:10217000035006E1030E005C0001D8B400D1020157
:10218000035006E1040E005C0001D8B40AD102013C
:10219000035006E1050E005C0001D8B41BD102011A
:1021A000035006E1060E005C0001D8B4B7D102016D
:1021B000035006E1070E005C0001D8B4C8D102014B
:1021C000035006E1080E005C0001D8B4D2D1020130
:1021D000035006E1090E005C0001D8B4EED1020103
:1021E000035006E10A0E005C0001D8B406D20201D9
:1021F000035006E10B0E005C0001D8B41ED20201B0
:10220000035006E1640E005C0001D8B435D202012F
:10221000800E035C05E100520001D8B43FD20201F8
:10222000035006E1650E005C0001D8B449D20201FA
:10223000035006E1660E005C0001D8B453D20201DF
:10224000035006E1670E005C0001D8B46CD20201B5
:10225000035006E1680E005C0001D8B477D2020199
:10226000035006E1690E005C0001D8B489D2020176
:10227000035006E16A0E005C0001D8B494D202015A
:10228000035006E16B0E005C0001D8B4ADD2020130
:10229000035006E16C0E005C0001D8B4B8D2020114
:1022A000035006E16D0E005C0001D8B4CAD20201F1
:1022B000035006E16E0E005C0001D8B4D5D20201D5
:1022C000035006E16F0E005C0001D8B4E7D20201B2
:1022D000035006E1700E005C0001D8B4F2D2020196
:1022E000035006E1710E005C0001D8B4FFD2020178
:1022F000035006E1720E005C0001D8B414D3020151
:10230000800E035C06E1010E005C0001D8B42ED300
:10231000020149D30101FA6B5B0EF96F0201056BF3
:10232000370E066F0001D7DE0201056B370E066F10
:102330000001D1DE4CD30101FA6B5B0EF96F020193
:10234000056B370E066F0001C6DE010E0201056F38
:10235000370E066F0001BFDE3AD30101FA6B5B0E48
:10236000F96F0201056B370E066F0001B4DE020E35
:102370000201056F370E066F0001ADDE28D30101A3
:10238000FA6B5B0EF96F0201056B370E066F0001E9
:10239000A2DE030E0201056F370E066F00019BDE01
:1023A00016D30101FA6B5B0EF96F0201056B370E54
:1023B000066F000190DE040E0201056F370E066FF6
:1023C000000189DE02C205F2370E0201066F00012C
:1023D00082DEFDD20101FA6B5B0EF96F0201056B23
:1023E000370E066F000177DE050E0201056F370E0E
:1023F000066F000170DE0101FA6B5F0EF96FE7C036
:1024000005F2370E0201066F000165DEE6C005F237
:10241000370E0201066F00015EDEE5C005F2370EE1
:102420000201066F000157DEE3C005F2370E02011C
:10243000066F000150DEE2C005F2370E0201066FA2
:10244000000149DEE1C005F2370E0201066F00010E
:1024500042DE0101FA6B6B0EF96FEBC105F2370E2C
:102460000201066F000137DEEAC105F2370E0201F4
:10247000066F000130DEE8C105F2370E0201066F7B
:10248000000129DEEDC105F2370E0201066F0001E1
:1024900022DEECC105F2370E0201066F00011BDEE1
:1024A000E9C105F2370E0201066F000114DEEFC12B
:1024B00005F2370E0201066F00010DDEEEC105F2D6
:1024C000370E0201066F000106DE0E0E0201056FD7
:1024D000370E066F0001FFDD0101FA6B7D0EF96F0B
:1024E000010E0201056F370E066F0001F4DD0201D7
:1024F000056B370E066F0001EEDD020E0201046F60
:10250000300E076F0001D6DD0201042FF9D7090E46
:10251000056F370E066F0001DEDD59D20101FA6B3F
:102520005B0EF96F0201056B370E066F0001D3DDFC
:10253000060E0201056F370E066F0001CCDD02C2E8
:1025400005F2370E0201066F0001C5DD40D2010120
:10255000FA6B5B0EF96F0201056B370E066F000117
:10256000BADD070E0201056F370E066F0001B3DDFD
:102570002ED20101FA6B5B0EF96F0201056B370E6B
:10258000066F0001A8DD080E0201056F370E066F09
:102590000001A1DD050E0201046F04510001F5ECFC
:1025A00000F00201042B006E076F000183DD090EAD
:1025B0000201045DF2E100010AD20101FA6B5B0E37
:1025C000F96F0201056B370E066F000184DD090EFD
:1025D0000201056F370E066F00017DDDF1C105F2C6
:1025E000370E0201066F000176DDF0C105F2370EED
:1025F0000201066F00016FDDEAD10101FA6B5B0E8B
:10260000F96F0201056B370E066F000164DD0A0EDB
:102610000201056F370E066F00015DDDF1C105F2A5
:10262000370E0201066F000156DDF0C105F2370ECC
:102630000201066F00014FDDCAD10101FA6B5B0E8A
:10264000F96F0201056B370E066F000144DD0B0EBA
:102650000201056F370E066F00013DDD0201056BBB
:10266000370E066F000137DD780E0201056F370E59
:10267000066F000130DDABD10101FA6B5B0EF96F23
:102680000201056B370E066F000125DD640E0201A5
:10269000056F370E066F00011EDD99D10101FA6B3F
:1026A0005B0EF96F800E0201056F370E066F000199
:1026B00012DD0201056B370E066F00010CDD87D1BC
:1026C0000101FA6B5B0EF96F0201056B370E066FA5
:1026D000000101DD650E0201056F370E066F000176
:1026E000FADC75D10101FA6B5B0EF96F01C205F2DC
:1026F000370E0201066F0001EEDC00C205F2370E54
:102700000201066F0001E7DCEBC105F2370E0201A2
:10271000066F0001E0DCEAC105F2370E0201066F28
:102720000001D9DC54D10101FA6B5B0EF96F01C2D3
:1027300005F2370E0201066F0001CDDC00C205F282
:10274000370E0201066F0001C6DC41D10101FA6BB0
:102750005B0EF96F01C205F2370E0201066F000130
:10276000BADC00C205F2370E0201066F0001B3DCCD
:10277000E8C105F2370E0201066F0001ACDC27D17B
:102780000101FA6B5B0EF96F01C205F2370E02010F
:10279000066F0001A0DC00C205F2370E0201066FD1
:1027A000000199DC14D10101FA6B5B0EF96F01C2D3
:1027B00005F2370E0201066F00018DDC00C205F242
:1027C000370E0201066F000186DCEDC105F2370EFF
:1027D0000201066F00017FDCECC105F2370E020139
:1027E000066F000178DCF3D00101FA6B5B0EF96F24
:1027F00001C205F2370E0201066F00016CDC00C257
:1028000005F2370E0201066F000165DCE0D0010120
:10281000FA6B5B0EF96F01C205F2370E0201066F0B
:10282000000159DC00C205F2370E0201066F0001FB
:1028300052DCE9C105F2370E0201066F00014BDCE4
:10284000C6D00101FA6B5B0EF96F01C205F2370EBB
:102850000201066F00013FDC00C205F2370E0201E3
:10286000066F000138DCB3D00101FA6B5B0EF96F23
:1028700001C205F2370E0201066F00012CDC00C216
:1028800005F2370E0201066F000125DCEEC105F2EC
:10289000370E0201066F00011EDC99D00101FA6BB0
:1028A0005B0EF96F01C205F2370E0201066F0001DF
:1028B00012DC00C205F2370E0201066F00010BDCCC
:1028C00086D00101FA6B5B0EF96F01C205F2370E7B
:1028D0000201066F00016BEC10F000C205F2370E2A
:1028E0000201066F00016BEC10F071D00101FA6B70
:1028F0005B0EF96F01C205F2370E0201066F00018F
:102900006BEC10F000C205F2370E0201066F0001F9
:102910006BEC10F0320E0201056F370E066F0001EE
:102920006BEC10F054D09886000E86B6010E0201B2
:10293000046F0101FA6B5B0EF96F01C205F2370EED
:102940000201066F00016BEC10F000C205F2370EB9
:102950000201066F00016BEC10F004C205F2370EA5
:102960000201066F00016BEC10F031D00101FA6B2F
:102970005B0EF96F800E0201056F370E066F0001C6
:102980006BEC10F0010E0201056F370E066F0001AF
:102990006BEC10F002C205F2370E0201066F000167
:1029A0006BEC10F014D00101FA6B5B0EF96F0201B1
:1029B000056B370E066F00016BEC10F0040E020180
:1029C000056F370E066F00016BEC10F000D0000CA5
:1029D00005C207F204C206F207C203F0020106C2F2
:1029E000E9FF07C2EAFFEF5206E0062BD8B4072B37
:1029F0000001F2D702010451065D006E055107592E
:102A0000036E00C001F0026E00010FEF15F002012D
:102A1000036B026B056B5B0E046F0001D9D702C01C
:102A200003F00150035205E101500201025D0DE285
:102A30000001036A020102515B0FE96E000E0320E0
:102A4000EA6EEF500327022BE5D7031F03C201F004
:102A5000000171EF15F0640E0201076F988086A0E7
:102A600004D0075302E00707F9D70651F2CF08F266
:102A7000F29E00014FEC00F0020108BFF28E956A51
:102A80008C6E96908D9000D096908D800001000CF9
:102A9000020103BF11D00F0E006E023900160A0E9C
:102AA000005C03E2300E002602D00351002600C075
:102AB00006F20001D0DF02010F0E02170A0E025DBE
:102AC00002E2300E02D0039F0351022702C206F237
:102AD0000001C1DF9AEF15F00201006B016B0001EC
:102AE00096D701C001F2020E0201066F0001B3DFAA
:102AF000036A020100515B0FE96E000E0320EA6ECB
:102B0000EF5212E0036A00515B0FE96E000E0320E2
:102B1000EA6EEFCF02F202C206F200019CDF020170
:102B2000002B0001E5D7020101C202F2370E036F4C
:102B30000001AED7030E0201066F00018CDF000C0E
:102B4000D56ACD6AADEC0EF09D9AF29AF29CF29E97
:102B5000F2BEFDD750EF17F094820A0E006E04000B
:102B6000002EFDD794800A0E006E0400002EFDD7C3
:102B70008B9294920A0E006E0400002EFDD78B906B
:102B8000949002010251FE0B056F0D6F0001F6ECEF
:102B90000CF002010D6B0001F6EC0CF0070E0201C7
:102BA0000325E96E000E0421EA6EEFCF05F205C29F
:102BB0000DF20001F6EC0CF0060E02010325E96EA1
:102BC000000E0421EA6EEFCF05F205C20DF20001FE
:102BD000F6EC0CF0050E02010325E96E000E04214F
:102BE000EA6EEF503F0B066F0D6F0001F6EC0CF034
:102BF000040E02010325E96E000E0421EA6EEFCFF8
:102C000005F205C20DF20001F6EC0CF0030E020114
:102C10000325E96E000E0421EA6EEFCF05F205C22E
:102C20000DF20001F6EC0CF0020E02010325E96E34
:102C3000000E0421EA6EEFCF05F205C20DF200018D
:102C4000F6EC0CF0010E02010325E96E000E0421E2
:102C5000EA6EEFCF05F205C20DF20001F6EC0CF0C2
:102C600094920000948082A0FED70A0E006E0400A9
:102C7000002EFDD700D0000094820A0E006E0400E2
:102C8000002EFDD74DEF16F0D00E0201026F01C2EB
:102C900004F200C203F200015FD7A1EF17F0F29C2B
:102CA000F29EF2BEFDD70201096B1C0E086F040EE6
:102CB0000A6F00015AEC0FF001C0FFF100C0FEF1F5
:102CC0000101FEC100F0FF51036E06E1020E005C3F
:102CD0000001D8B4BAD00101035006E1030E005C34
:102CE0000001D8B4BCD00101035006E1070E005C1E
:102CF0000001D8B4C5D00101035006E1640E005CA8
:102D00000001D8B4D6D00101035006E1050E005CE5
:102D10000001D8B420D10101035006E1650E005C2A
:102D20000001D8B422D10101035006E1060E005C77
:102D30000001D8B407D20101035006E1080E005C7F
:102D40000001D8B42AD20101035006E1090E005C4B
:102D50000001D8B42CD20101035006E1660E005CDC
:102D60000001D8B444D20101035006E1670E005CB3
:102D70000001D8B447D20101035006E1680E005C9F
:102D80000001D8B460D20101035006E1690E005C75
:102D90000001D8B463D20101035006E16A0E005C61
:102DA0000001D8B471D20101035006E16B0E005C42
:102DB0000001D8B474D20101035006E16C0E005C2E
:102DC0000001D8B48FD20101035006E16D0E005C02
:102DD0000001D8B493D20101035006E16E0E005CED
:102DE0000001D8B4A2D20101035006E16F0E005CCD
:102DF0000001D8B4A6D20101035006E1700E005CB8
:102E00000001D8B4AAD20101035006E1710E005CA2
:102E10000001D8B4C1D20101035006E1720E005C7A
:102E20000001D8B4C5D20101035006E1730E005C65
:102E30000001D8B4C9D20101035006E1740E005C50
:102E40000001D8B4E8D2010105D30201016B020EE2
:102E5000006F026B00018EEC10F03EDE06D3020123
:102E6000016B030E006F026B00018EEC10F034DE7C
:102E7000640E0201006F00014BEC02F0FF00F5D27E
:102E8000F29CF29EF2BEFDD70201016B070E006FAD
:102E9000026B00018EEC10F01FDEADEC0EF050D690
:102EA000640E0201006F00014BEC02F000EF5BF0DA
:102EB000DCD20201096B200E086F020E0A6F0001BE
:102EC0005AEC0FF000C0E7F00201096B220E086F08
:102ED000020E0A6F00015AEC0FF000C0E6F002018A
:102EE000096B240E086F020E0A6F00015AEC0FF0F6
:102EF00000C0E5F00201096B260E086F020E0A6F92
:102F000000015AEC0FF000C0E3F00201096B280E3B
:102F1000086F020E0A6F00015AEC0FF000C0E2F0D9
:102F20000201096B2A0E086F020E0A6F00015AECAB
:102F30000FF000C0E1F00201016BE00E006F000134
:102F4000A3D60201016B640E006F026B00018EECD0
:102F500010F0C2DD8AD20201016B050E006F026B18
:102F600000018EEC10F0B8DD80D2D8511508D8B031
:102F7000DFD00201096B200E086F040E0A6F0001FA
:102F80005AEC0FF001C0EBF100C0EAF10201096B4D
:102F9000240E086F020E0A6F00015AEC0FF000C0F9
:102FA000E8F10201096B260E086F040E0A6F00019A
:102FB0005AEC0FF001C0EDF100C0ECF10201096B19
:102FC0002A0E086F020E0A6F00015AEC0FF000C0C3
:102FD000E9F10201096B2C0E086F040E0A6F000163
:102FE0005AEC0FF001C0EFF100C0EEF10201006BEE
:102FF000EBC102F2EAC101F2000194EC0EF0020E04
:103000000201006FEDC102F2ECC101F2000194EC8B
:103010000EF00101EEC100F0EF51036E05E1C80EA4
:10302000005C00012AE00101010E035C05E1900E45
:10303000005C000130E00101020E035C05E1580E66
:10304000005C000137E00101030E035C05E1200E86
:10305000005C00013EE00101030E035C05E1E80EA7
:10306000005C000145E00101070E035C05E1D00EA4
:10307000005C00014DE001015BD00101EF6BC80E67
:10308000EE6F0001E96B3C0EE86FF70EEB6FDC0EA4
:10309000EA6F01014DD0010E0101EF6F900EEE6F4E
:1030A0000001E96B780EE86FFB0EEB6FEE0EEA6F36
:1030B00001013ED0020E0101EF6F580EEE6F0001CC
:1030C000E96BB40EE86FFD0EEB6F490EEA6F01017C
:1030D0002FD0030E0101EF6F200EEE6F0001E96BA0
:1030E000F00EE86FFD0EEB6FF70EEA6F010120D0D6
:1030F000030E0101EF6FE80EEE6F010E0001E96FA4
:103100002C0EE86FFE0EEB6F5F0EEA6F010110D020
:10311000070E0101EF6FD00EEE6F020E0001E96F96
:10312000580EE86FFF0EEB6F2F0EEA6F010100D013
:103130000201016B650E006F026B00018EEC10F056
:10314000CBDC93D10201096B200E086F020E0A6FCF
:1031500000015AEC0FF0005206E1015204E1025264
:1031600002E103520CE0010E0101E66F0201016B66
:10317000DA0E006F00015FEC02F0F28A03D0010169
:10318000E66BF29A0201016B060E006FE6C102F2D5
:1031900000018EEC10F0A0DC68D10201016B080E7A
:1031A000006F026B00018EEC10F096DC5ED1020124
:1031B000096B200E086F040E0A6F00015AEC0FF025
:1031C00001C0FFF100C0FEF10101FE3D03D0FF3D53
:1031D00001D004D0FFC1F1F1FEC1F0F10201016B99
:1031E000090E006F026B00018EEC10F075DCFFC160
:1031F00001F2FEC100F20201026B00018EEC10F040
:103200006BDC33D10201096B200E086F040E0A6FCC
:1032100000015AEC0FF001C0EBF100C0EAF102012D
:10322000006BEBC102F2EAC101F2000194EC0EF076
:10323000FFC101F2FEC100F20201026B00018EEC3F
:1032400010F04ADC12D1FFC101F2FEC100F202010E
:10325000026B00018EEC10F03FDC07D10201096B1C
:10326000200E086F020E0A6F00015AEC0FF000C02A
:10327000E8F1FFC101F2FEC100F20201026B0001A0
:103280008EEC10F029DCF1D0FFC101F2FEC100F29A
:103290000201026B00018EEC10F01EDCE6D0020190
:1032A000096B200E086F040E0A6F00015AEC0FF034
:1032B00001C0EDF100C0ECF1020E0201006FEDC1A2
:1032C00002F2ECC101F2000194EC0EF0FFC101F238
:1032D000FEC100F20201026B00018EEC10F06CECFA
:1032E00015F0C3D0FFC101F2FEC100F20201026B72
:1032F00000018EEC10F06CEC15F0B7D00201096BF8
:10330000200E086F020E0A6F00015AEC0FF000C089
:10331000E9F1FFC101F2FEC100F20201026B0001FE
:103320008EEC10F06CEC15F0A0D0FFC101F2FEC1E4
:1033300000F20201026B00018EEC10F06CEC15F053
:1033400094D0FFC101F2FEC100F20201026B000144
:103350008EEC10F06CEC15F088D00201096B200E99
:10336000086F020E0A6F00015AEC0FF000C0F4F172
:103370000101F45303E098948F8402D098948F94C1
:10338000FFC101F2FEC100F20201026B00018EECEE
:1033900010F06CEC15F069D0FFC101F2FEC100F233
:1033A0000201026B00018EEC10F06CEC15F05DD0A8
:1033B000FFC101F2FEC100F20201026B00018EECBE
:1033C00010F06CEC15F051D00201096B200E086F63
:1033D000020E0A6F00015AEC0FF000C0F6F1988659
:1033E0000101F76B86B6F72BF56BFA6B5B0EF96F85
:1033F000FFC105F2370E0201066F00016BEC10F001
:10340000FEC105F2370E0201066F00016BEC10F0F1
:103410006CEC15F02AD00101FA6B5B0EF96FFFC15D
:1034200005F2370E0201066F00016BEC10F0FEC1D1
:1034300005F2370E0201066F00016BEC10F0F6C1C9
:1034400005F2370E0201066F00016BEC10F06CEC18
:1034500015F00BD00201016B010E006F026B000131
:103460008EEC10F06CEC15F000D0ADEC0EF0C00E50
:10347000F212C0EF1AF00201026B016B006B0151F6
:103480000101FF5D24E308E1FE510201005DD8A0C7
:1034900002D001011CD001015B0E02010025E96E82
:1034A000000E0121EA6EEFCF05F205C206F200011F
:1034B0002BEC15F05B0E02010025E96E000E0121D8
:1034C000EA6EEF500227002BD8B4012BD8D70201A7
:1034D000021F0239006E0F0E00160050300F036FEE
:1034E00002510F0B300F046F0351390802E2070E2F
:1034F00003270451390802E2070E042703C206F22B
:1035000000012BEC15F004C206F22BEC15F0030EB3
:103510000201066F00012BEC15F0000CF86AD09E3A
:103520000D8EEA6AE96A7E86110EAF6E040E7F6E1A
:10353000A60EAC6E900EAB6EC150C00B0F09C16EE3
:10354000070EB46E196A1A6A010E0101F06FF16B71
:10355000F26FF36BF56BF66BF96BFA6B0001B0EF82
:103560000EF0988286B208D0F29CF29EF2BEFDD791
:103570001AEF10F0C00EF212D7A102D04FEF16F0E2
:103580000101E23D06D0E35304E1E45302E1E553D7
:1035900052E0E22D24D0E35322E1E45320E1E5534D
:1035A0001EE10201016B0B0E006F026B00018EEC3D
:1035B00010F06CEC15F0EA6A5B0EE96EE26AF00E50
:1035C000E16E780E016EE6CFEEFF012EFCD7010111
:1035D000FF6B780EFE6F00014EDF27D00101E25134
:1035E000020824E1E35322E1E45320E1E5531EE124
:1035F0000201016B0B0E006F026B00018EEC10F0EC
:103600006CEC15F0EA6A5B0EE96E010EE26E680E74
:10361000E16E780E016EE6CFEEFF012EFCD70101C0
:10362000FF6B780EFE6F000126DF0101E56BE46B96
:10363000E36BFF0EE26F938081B00AD0640E02014B
:10364000006F00014BEC02F0938081B000D00101CB
:10365000F65325E09886F86B86B6F82BF751F85D9F
:103660001DE0F52BF551320818E2F8C1F7F1F853D7
:1036700002E0F6B104D0F85310E1F6A30ED0800EAC
:103680000201016F010E006FF8C102F200018EEC21
:1036900010F06CEC15F00101F56B01D0F56B000139
:0436A00060D70300EC
:020000040030CA
:0E00000000260C1E838381000FC00FE00F400E
:00000001FF
